S027000062696E2F64656D6F70726F675F6E75636C656F5F73746D33326631303372622E737265636D
S315080060006C01002049630008096600080966000853
S315080060100966000809660008096600080966000896
S315080060200966000809660008096600080966000886
S31508006030096600080966000809660008F965000887
S315080060400966000809660008096600080966000866
S315080060500966000809660008096600080966000856
S315080060600966000809660008096600080966000846
S315080060700966000809660008096600080966000836
S315080060800966000809660008096600080966000826
S315080060900966000809660008096600080966000816
S315080060A00966000809660008096600080966000806
S315080060B009660008096600080966000809660008F6
S315080060C009660008096600080966000809660008E6
S315080060D009660008096600080966000809660008D6
S315080060E009660008096600080966000809660008C6
S315080060F009660008096600080966000809660008B6
S3150800610009660008096600080966000809660008A5
S315080061100966000809660008096600080966000895
S315080061200966000809660008096600080966000885
S315080061300966000809660008096600080966000875
S315080061400966000809660008096600080966000865
S31508006150EE11AA5510B504464FF48840C4F2000063
S31508006160202146F6E903C0F60003984701280BD11B
S315080061704FF48840C4F2000046F6E103C0F6000377
S3150800618098472070012010BD002010BD70B586B05C
S315080061904FF40030012146F2C973C0F60003984750
S315080061A00520012146F2A573C0F600039847182377
S315080061B08DF807300426ADF8046003238DF8063001
S315080061C04FF40065C4F2010528460DEB060146F2B8
S315080061D00D64C0F60004A0478DF807600823ADF8E3
S315080061E0043028460DEB0601A0474FF4614302939D
S315080061F00023ADF80C30ADF80E30ADF81030ADF820
S3150800620014300C23ADF812304FF48844C4F200045D
S31508006210204602A946F2ED73C0F6000398472046C9
S31508006220012146F6C503C0F60003984706B070BDBF
S315080062304FF46D42CEF20002D16801F4E061042306
S31508006240C0F2FA530B43D360BFF34F8FFEE700BF8C
S3150800625008B540F25903C2F200031B7843BB40F26B
S315080062601400C2F2000046F25513C0F60003984720
S31508006270012865D140F21403C2F200031B78002BF3
S315080062805ED046F2ED53C0F60003984740F25C0331
S31508006290C2F20003186040F25903C2F20003012259
S315080062A01A7040F25803C2F2000300221A7008BDA1
S315080062B040F25803C2F200031878224B184446F2FB
S315080062C05513C0F600039847012826D140F2580313
S315080062D0C2F200031A780132D2B21A7040F21403DD
S315080062E0C2F200031B7893422AD140F25903C2F244
S315080062F0000300221A7040F21403C2F200035B780E
S31508006300FF2B1DD140F21403C2F200039B78BBB9E0
S3150800631046F23123C0F60003984746F2ED53C0F61D
S315080063200003984740F25C03C2F200031B6864331B
S31508006330984281BF40F25903C2F2000300221A7044
S3150800634008BD00BF1500002010B517498D4640F25C
S315080063500002C2F2000240F21403C2F200039A429B
S3150800636010D2131D0F4CE41A24F00304043400233E
S31508006370104646F6F401C0F600015A581A5004337E
S31508006380A342FAD109480A494FF000028842B8BF29
S3150800639040F8042BFADB46F27143C0F6000398472F
S315080063A010BD00BF170000206C010020140000205B
S315080063B06C00002000B583B00420012146F2A573C5
S315080063C0C0F6000398472023ADF8043003238DF860
S315080063D0063010238DF807304FF40060C4F2010030
S315080063E001A946F20D63C0F60003984703B05DF8AD
S315080063F004FB00BF10B546F2ED53C0F600039847FC
S31508006400044640F26003C2F200031B68C31AB3F5E0
S31508006410FA7F2BD340F26403C2F200031B7883B9D8
S3150800642040F26403C2F2000301221A704FF40060BE
S31508006430C4F20100202146F2B163C0F60003984772
S315080064400FE040F26403C2F2000300221A704FF410
S315080064500060C4F20100202146F2B563C0F60003CD
S31508006460984740F26003C2F200031C6010BD00BFEB
S3150800647000B583B00023009301934FF48053C4F210
S3150800648002031A6842F001021A6059680022CFF620
S31508006490FF020A405A601A6822F0847222F4803297
S315080064A01A601A6822F480221A605A6822F4FE02D8
S315080064B05A604FF41F029A601A6842F480321A60D2
S315080064C04FF48053C4F2020340F2DC511A6802F416
S315080064D000320192009A01320092019A12B9009A8A
S315080064E08A42F3D14FF48053C4F202031B6813F4B3
S315080064F0003F00D1FEE74FF40053C4F202031A68C6
S3150800650042F010021A601A6822F003021A601A682A
S3150800651042F002021A604FF48053C4F202035A682A
S315080065205A605A6842F400525A605A6842F48062C5
S315080065305A605A6822F47C125A605A6842F4E81281
S315080065405A601A6842F080721A604FF48053C4F297
S3150800655002031A6812F0007FFBD04FF48053C4F28E
S3150800656002035A6822F003025A605A6842F002028D
S315080065705A604FF48053C4F202035A6802F00C02C0
S31508006580082AFAD146F2B533C0F60003984746F210
S31508006590B953C0F60003984746F28D13C0F60003B8
S315080065A0984746F2F535C0F6000546F25124C0F67E
S315080065B00004A847A047FCE74EF21003CEF20003FA
S315080065C041F63F12C0F201025A604FF46D42CEF214
S315080065D00002F02182F8231000229A600721196030
S315080065E040F26803C2F200031A60704740F268037B
S315080065F0C2F200031868704740F26803C2F200034B
S315080066001A6801321A607047FEE700BF2DE9F001EB
S31508006610CB7803F00F0513F0100F1CBF8B781D43C2
S315080066200B78F3B10768002301264FF00F0C06FA22
S3150800663003F20C88144094420FD19A000CFA02F81F
S3150800664027EA080705FA02F21743CA78282A08BF74
S31508006650446102D0482A08BF04610133082BE6D1F9
S3150800666007600B88FF2B20D94768002301264FF0C7
S315080066700F0C03F1080206FA02F20C881440944241
S315080066800FD19A000CFA02F827EA080705FA02F26F
S315080066901743CA78282A08BF4461CA78482A08BF17
S315080066A004610133082BE4D14760BDE8F001704767
S315080066B0016170474161704710B44FF48053C4F2CA
S315080066C002035B6803F00C03042B08D0082B0CD0DC
S315080066D09BBB4FF49053C0F27A03036032E04FF449
S315080066E09053C0F27A0303602CE04FF48053C4F24F
S315080066F002035A685B68C2F38342023213F4803F8E
S3150800670007D14FF41063C0F23D0303FB02F20260A7
S3150800671018E04FF48053C4F202035B6813F4003F99
S3150800672019BF4FF41063C0F23D034FF49053C0F203
S315080067307A0303FB02F2026004E04FF49053C0F2BE
S315080067407A0303604FF48053C4F202035968C1F315
S31508006750031140F20402C2F20002515CC9B2046895
S3150800676024FA01F141605C68C4F30224145DE4B2C2
S3150800677021FA04F484605C68C4F3C224125DD2B2C0
S31508006780D140C1605A68C2F3813240F20003C2F2B6
S3150800679000039B5CDBB2B1FBF3F101615DF8044BCE
S315080067A0704700BF39B14FF48053C4F202039A69A7
S315080067B01043986170474FF48053C4F202039A69F4
S315080067C022EA00009861704739B14FF48053C4F249
S315080067D00203DA691043D86170474FF48053C4F254
S315080067E00203DA6922EA0000D861704730B587B03B
S315080067F004460D46038A23F440531B041B0CCA881F
S315080068001343038283890989AA880A4369890A4343
S3150800681023F4B05323F00C031B041B0C13439BB245
S315080068208381838A23F440731B041B0CAA891343B0
S31508006830838201A846F2B963C0F6000398474FF46D
S315080068406053C4F201039C420CBF049A039AA389BD
S315080068501BB2002B02EB820202EB8202BDBF2B6841
S315080068605B00B2FBF3F22968A4BF8900B2FBF1F220
S3150800687048F21F53C5F2EB13A3FB02135B091D0174
S31508006880642003FB1023A08900B200280BDADB0082
S31508006890323348F21F51C5F2EB11A1FB0321C1F3B4
S315080068A0421129430AE01B01323348F21F51C5F24F
S315080068B0EB11A1FB0321C1F34311294389B22181BD
S315080068C007B030BD29B183899BB243F40053838155
S315080068D07047838923F400531B041B0C838170477C
S315080068E08088C0F308007047038819420CBF00204F
S309080068F001207047BE
S315080068F4020406080000000001020304010203045E
S309080069040607080963
S7050800600092
